:1000000000308A00E9290000FF00030E8301A100EF
:100010007F08A0000A08A8008A01A00E0408A20018
:100020007708A3007808A4007908A5007A08A6003C
:100030007B08A700831383128B1E20280B193328FB
:10004000220884002308F7002408F8002508F90096
:100050002608FA002708FB0028088A00210E8300E2
:10006000FF0E7F0E0900AA0A0319AB0A2A08423CB8
:10007000031DE2282B080F3C031DE228AB01AA0157
:10008000AC0A0319AD0AAD08031D4A282C083B3CF5
:1000900003184F28AE0A0319AF0AAD01AC01401E88
:1000A000E2282030C00605303007C3003108C40004
:1000B0000318C40A44083902031C6428031D972846
:1000C00038084302031C972805303207C50033085F
:1000D000C6000318C60A46083B02031C7528031D08
:1000E00097283A084502031C972805303407C700B3
:1000F0003508C8000318C80A48083D02031C8628B2
:10010000031D97283C084702031C97280530360733
:10011000C9003708CA000318CA0A4A083F02031C6C
:100120009828031D97283E0849020318982840176D
:10013000401BC6283008B8070318B90A3108B907A8
:100140000310B90CB80C3208BA070318BB0A3308FD
:10015000BB070310BB0CBA0C3408BC070318BD0A5C
:100160003508BD070310BD0CBC0C3608BE070318CC
:10017000BF0A3708BF070310BF0CBE0CB101B001A6
:10018000B301B201B501B401B701B601B908031D4D
:10019000CD283808053C0318E128BB08031DD428E6
:1001A0003A08053C0318E128BD08031DDB283C087C
:1001B000053C0318E128BF08031DE2283E08053C62
:1001C000031840170B118A112028AB01AA01AD01B9
:1001D000AC01AF01AE014012C0124013A901831659
:1001E0000108C73908388100831290010030F800F7
:1001F000920000308316920083128B16C0308B045D
:100200008316811300306500F0306600850183128B
:1002100085018316860183128601F029AF01AE01A4
:10022000AD01AC01C01240134012A901B101B001EF
:10023000B301B201B501B401B701B601B90106308D
:10024000B800BB01BA00BD01BC00BF01BE008316EF
:10025000061683124010061A40148316861683125F
:10026000C010861AC0148316061783124011061B8D
:100270004015831686178312C011861BC01583167E
:1002800005118312051583160510831205148316B4
:1002900085108312851440160034831605118312CD
:1002A000051183168510831285104012AF01AE012F
:1002B000AD01AC01003442308400000803196F29FD
:1002C0000130F800F701F70B6329F80B62294A3077
:1002D000F700F70B692900000000800B60298629D0
:1002E000401F7429A90A40132908023C03189029C9
:1002F0004D218316051083120510831685100230D8
:1003000083128506C100FA30C2005B29C10B832924
:1003100083168615831286198F290E2190297D292F
:10032000003040180130C1008316061600308312D9
:10033000061A013041020319A629B00A0319B10AAD
:100340008316061683124010061A40140030C01897
:100350000130C1008316861600308312861A0130E0
:1003600041020319BC29B20A0319B30A831686167F
:100370008312C010861AC014003040190130C10029
:100380008316061700308312061B01304102031941
:10039000D229B40A0319B50A83160617831240112D
:1003A000061B40150030C0190130C10083168617A6
:1003B00000308312861B013041020319E829B60A76
:1003C0000319B70A831686178312C011861BC0153E
:1003D000092A84011F30830507309F00A901E52801
:1003E0008316051083120514831686158312861949
:1003F000FF29831686158312861DF9290E21C01A3E
:10040000032A8510042A8514831685108312401A46
:1004100070292F08043C0318182AFF3A031D142AD8
:100420002E089F3C0318182A401A182A0E21222A47
:10043000AF08031D1F2A2E08043C0318222A401E61
:08044000222A4D21F42963007A
:02400E00693F08
:00000001FF
